:020000040000FA
:10000000700ED36E9B8CAAD1FACF0BF087EF00F065
:080018000E6ED8CF0FF0E0CF0F
:100020000DF0FACF0CF0F950F2B409D09EA802D02E
:100030009DB8E6D09EAA02D09DBAA9D0FF00896AD9
:10004000926AF294442A400E446402D0010E446E37
:10005000486A44504560488446604882476048800A
:100060008A6A8B50F80B481009B0070A8B6E8DEC2A
:1000700001F0FF0E926E896EF9501A50F92636D0B3
:100080002ED026D01ED016D00ED006D01A6A800EE2
:100090008A6E321C926E32D00E0E1A6E400E8A6E2E
:1000A000311C926E2BD00C0E1A6E200E8A6E301CF4
:1000B000926E24D00A0E1A6E100E8A6E2F1C926E4B
:1000C0001DD0080E1A6E080E8A6E2E1C926E16D067
:1000D000060E1A6E040E8A6E2D1C926E0FD0040E40
:1000E0001A6E020E8A6E2C1C926E08D02CEC01F057
:1000F000020E1A6E010E8A6E2B1C926E0DC0E0FF6E
:100100000F38D86E0E3A0E380CC0FAFF1000F950B6
:100110009E92397039B038D03A663A06CEEC0CF07F
:10012000E86620D060A41ED05D5002620CD05C5006
:10013000036209D00830010B376E010E081437181E
:1001400002E1609E0FD05D5004620CD05C500562ED
:1001500009D00830E830010B376E010E081437184B
:1001600001E1608E644E07D0020E64620DD08250B1
:10017000300B636E09D074EC01F0030E646E825094
:10018000300B636201D0626E0BC0FAFF11009E9AC1
:10019000ABA205D0AB98AE50AE50AE50AB88ABA47E
:1001A00002D0AE50ABD7D624696E65B4A7D765B080
:1001B00005D0AE50CC0AA2E16580A0D765B207D0C9
:1001C000AE50F00A01E09AD76582676A97D711EEC0
:1001D00000F06750AECFE3FF672A100E67628ED73C
:1001E0006584676A65906592F29E010EFC6E7C0ED6
:1001F000FD6E050EFE6E000EFF6EF950F28E1000C1
:1002000065B60DD011EE10F06A50E350ACA2FED7E7
:10021000AD6E6A2A1B0E6A6271D765866FD76596C6
:100220006A6AAC9AF29E68B007D0658EFF0E116EB6
:10023000126E136E658A05D0D6CF01F069C000F04A
:10024000659E010EFC6EC40EFD6E040EFE6E000E69
:10025000FF6EF28EF9501000406611D01BC02BF0DB
:100260001CC02CF01DC02DF01EC02EF01FC02FF0A2
:1002700020C030F021C031F022C032F012003F2EF9
:1002800008D03EC03FF0422E04D040C042F041664C
:1002900041063F50415CE2E623C02BF024C02CF025
:1002A00025C02DF026C02EF027C02FF028C030F03A
:1002B00029C031F02AC032F012001BC023F01CC04C
:1002C00024F01DC025F01EC026F01FC027F020C05E
:1002D00028F021C029F022C02AF03EC041F03EC0E3
:1002E0003FF040C042F0120057B0120057A2120077
:1002F00049C04CF04AC04DF04BC04EF04FC049F0E1
:1003000050C04AF051C04BF054C053F054C055F0A7
:1003100052C056F0579257801200526608D057903C
:1003200049C045F04AC046F04BC047F01200552E78
:100330000BD054C055F0562E07D052C056F053661D
:1003400002D0579001D053065550535CE9E64CC09B
:1003500045F04DC046F04EC047F0120000EE00F0F0
:10036000EE50002600B0012AEAA0FAD700EE00F015
:10037000006602D0450E006E016602D0300E016E9E
:10038000AEEC0CF069EC0EF00A50AA0A0EE0AEECEE
:100390000CF00C0E026E0B0E046EF90E076E050EBD
:1003A000086E036A056A066A096AC26A0F0EC16EA0
:1003B000070EB46EFF0E926E896E936AF00E946E05
:1003C0008A6A8B6A010E406E0C0E3E6E050E526EEE
:1003D000400E546E0C0E5D6E5C6A5B6A5A6A088051
:1003E000300E626E636E050E646E686AC00ED56E66
:1003F000D66ACA6ACC6A4B0ECA6E07C0CBFFCA84E3
:10040000080EB86E460EAF6E100EB06E040EAC6ED7
:10041000900EAB6EF26A9D6AA06A9E6AF06AC00E88
:10042000F16E020E9F6ED08E9D829F9A9F989D883E
:100430009D8AE00EF26E82BA20D082B815D0080EE6
:10044000216E0C0E026E046E036A056A066AF90ECE
:10045000076E086A096A0A6A5DEC0EF005EC18F08E
:10046000300E6262FDD7FF00800E216E09805BECCA
:100470000EF005EC18F082AAFCD7FF0E1B6E1C6E66
:100480001D6E1E6E1F6E206E216E226E5DEC01F0E1
:10049000010EB8EC0CF0640E44EC0CF0020EB8EC5B
:1004A0000CF0640E44EC0CF0030EB8EC0CF0640E8F
:1004B00044EC0CF0FA0E44EC0CF07FEC0CF0640E03
:1004C00044EC0CF07FEC0CF0406A436A18C019F061
:1004D00017C018F016C017F015C016F014C015F0AC
:1004E00013C014F012C013F011C012F010C011F0BC
:1004F0003A0E736E000E93EC1BF0106E105065BA3E
:100500001BD0116201D0F4D7126201D0F1D713626F
:1005100001D0EED7146201D0EBD7156201D0E8D735
:10052000166201D0E5D7176201D0E2D7186201D078
:10053000DFD7196201D0DCD7659A070E736E010E02
:1005400093EC1BF0336E210E736E070E93EC1BF0D1
:100550003B6E65BC09D001500024D6240F0B346ECD
:100560000C0E3460C2EF1FF060BEEFEF05F0F950E3
:10057000070EFA6E1050040DF350C2D0658C9D9892
:1005800001EE00F0EECF34F0EECF35F029EC03F0C1
:10059000686E6B6EEECF34F0EECF35F029EC03F0E1
:1005A0006C6E6B263F0E6C6052D0EECF34F0EECF07
:1005B00035F029EC03F06D6E6B26EECF34F0EECF04
:1005C00035F029EC03F06E6E6B26EECF34F0EECFF3
:1005D00035F029EC03F06F6E6B26EECF34F0EECFE2
:1005E00035F029EC03F0706E6B26EECF34F0EECFD1
:1005F00035F029EC03F0716E6B26EECF34F0EECFC0
:1006000035F029EC03F065946B1821E16CC010F013
:100610006DC03BF06EC033F06FC001F070C000F0F1
:10062000609E71BE608E7FEC0CF068B007D0658E66
:10063000FF0E116E126E136E658A44D768A006D045
:10064000D6CF01F069C000F0659E3CD7FF006594ED
:1006500039D73430010B34B6020934BA040934BE38
:10066000080935B2100935B6200935BA400935BE3A
:0406700080091200EB
:10070000F92601EF04F02FEF04F082EF04F0CDEFB3
:1007100004F0F6EF04F0FFEF04F020EF05F03FEFF8
:1007200005F046EF05F06FEF05F087EF05F0AAEF53
:1007300005F0E4EF05F0EFEF05F0F8EF05F016EF48
:1007400006F03EEF06F055EF06F06DEF06F08BEF8A
:1007500006F051EF07F024EF08F02BEF08F032EF2E
:1007600008F039EF08F022EF09F086EF0AF08DEF7C
:100770000AF09EEF0AF0A5EF0AF0ACEF0AF0CEEF18
:100780000AF0EAEF0AF0F1EF0AF000EF0BF007EFE2
:100790000BF028EF0BF033EF0BF03EEF0BF056EFC2
:1007A0000BF097EF0BF0A3EF0BF0BFEF0BF0CBEFDD
:1007B0000BF0D2EF0BF0D9EF0BF0E4EF0BF0EBEF17
:1007C0000BF0F2EF0BF0F9EF0BF000EF0CF007EF8E
:1007D0000CF00EEF0CF015EF0CF01CEF0CF023EF0B
:1007E0000CF02FEF0CF036EF0CF03DEF0CF062EF59
:1007F00002F062EF02F062EF02F062EF02F062EFED
:1008000002F0460E736E140E93EC1BF0336E050E61
:10081000736E010E93EC1BF0406E526E5DEC01F0B6
:1008200068EC0CF000C01BF001C01CF068EC0CF090
:1008300000C01DF001C01EF068EC0CF000C01FF0FD
:1008400001C020F068EC0CF000C021F001C022F0E3
:10085000B4EC0CF062EC1BF0332EE0D733D6526AC6
:10086000040E406E5DEC01F0FF0E1B6E1C6E1D6EE3
:100870001E6E1F6E206E216E226EB4EC0CF0C8EC62
:100880000CF0090E526EE86AB8EC0CF0030E736EB1
:10089000010E93EC1BF0406E00EE1BF068EC0CF0C8
:1008A000070E0014E92668EC0CF0070E0114356EF3
:1008B000FE0E366E355204E036463650352EFCD7E5
:1008C0005DEC01F0EFCF36F0EF163650EF6204D05A
:1008D000002AD8B0012AE0D762EC1BF01B66DCD7F7
:1008E0001C66DAD71D66D8D71E66D6D71F66D4D742
:1008F0002066D2D72166D0D72266CED7640E44ECCC
:100900000CF0E0D5090E526E640E44EC0CF0030EB0
:10091000736E010E93EC1BF0406E00EE1BF068EC62
:100920000CF0070E0014E92668EC0CF0070E011419
:10093000356E010E366E3552D8B404D03646365078
:10094000352EFCD75DEC01F0EFCF36F0EF123650CC
:10095000EF6204D0002AD8B0012ADFD762EC1BF086
:10096000FF0E1B18DAE1FF0E1C18D7E1FF0E1D1851
:10097000D4E1FF0E1E18D1E1FF0E1F18CEE1FF0ECD
:100980002018CBE1FF0E2118C8E1FF0E2218C5E1A7
:10099000B4EC0CF0C8EC0CF095D53C0E736E0F0E59
:1009A00093EC1BF0336E100E736E070E93EC1BF07E
:1009B0003B6E00EE1BF068EC0CF0070E0014E9260D
:1009C00068EC0CF0070E0114356E010E366E3552D0
:1009D000D8B404D036463650352EFCD7EF6E3B5097
:1009E00044EC0CF0EF6A332EE4D76CD54380406AB8
:1009F000310E776E100E766E040E30EF1BF0030E84
:100A0000736E010E93EC1BF0526E406E3B5044EC43
:100A10000CF05DEC01F0FF0E1B6E1C6E1D6E1E6E69
:100A20001F6E206E216E226EB4EC0CF03B5044EC35
:100A30000CF05DEC01F07FEC0CF0332EE7D742D5E3
:100A40007FEC0CF0030E736E010E93EC1BF0336E13
:100A5000070E356EEA6A1B0EE96E010E366E01D086
:100A600036463650EF6E080E44EC0CF0EF6A36AEA8
:100A7000F7D7E92A352EF1D7332EEAD723D5310E11
:100A8000776E600E766E040E30EF1BF0070E736EFD
:100A9000010E93EC1BF0406E010E526E68EC0CF0F0
:100AA000070E0114F66E300EF76E08005DEC01F0D3
:100AB000F5501B6E1C6E1D6E1E6E1F6E206E216E1D
:100AC000226E030EF66402D0E86A02D0F650010FDF
:100AD000B8EC0CF062EC1BF0332EE0D7F3D4090E27
:100AE000526E030E406E5DEC01F07FEC0CF03B505B
:100AF00044EC0CF0356A5DEC01F0B4EC0CF08FECDA
:100B00000CF03B5044EC0CF0332EE9D7DBD4140E40
:100B1000736E080E93EC1BF0336E0C0E736E070EA3
:100B200093EC1BF03B6E010E366E01D036465DEC49
:100B300001F036501B6E1C6E1D6E1E6E1F6E206EF9
:100B4000216E226E3B5044EC0CF036AEEFD7332EC4
:100B5000EAD7B8D47FEC0CF0800E216E3B5044EC09
:100B60000CF07FEC0CF0800E226E3B5044EC0CF04D
:100B70007FEC0CF0800E1E6E3B5044EC0CF07FECD2
:100B80000CF0800E206E3B5044EC0CF07FEC0CF02F
:100B9000800E1F6E3B5044EC0CF0332EDBD77FEC05
:100BA0000CF0060E526E040EB8EC0CF0800E216EA6
:100BB000226E1E6E206E1F6EC8EC0CF0E86AB8EC58
:100BC0000CF0C8EC0CF07ED4010E526EB4EC0CF0BC
:100BD000310E776E380E766E040E30EF1BF07FEC20
:100BE0000CF0C80E44EC0CF065ACC2EF1FF06AD4F8
:100BF0007FEC0CF0050E736E000E93EC1BF0406E54
:100C0000010E366E01D036465DEC01F036501B12F7
:100C10001C121D121E121F1220122112221262EC2F
:100C20001BF036AEF0D7332EE3D74CD4060E526EFF
:100C3000030E736E000E93EC1BF0406EF66E300EDA
:100C4000F76E09005DEC01F0F5501B6E1C6E1D6E19
:100C50001E6E1F6E206E216E226EB4EC0CF0C80E5C
:100C600044EC0CF0C80E44EC0CF05DEC01F07FECB1
:100C70000CF0320E44EC0CF062EF02F07FEC0CF062
:100C8000060E526E68EC0CF0030E0114406E5DEC23
:100C900001F0356A8FEC0CF0B4EC0CF03B5044ECF6
:100CA0000CF0332EF9D762EF02F07FEC0CF0060E59
:100CB000526E68EC0CF0030E0114406E5DEC01F016
:100CC000080E356E8FEC0CF0B4EC0CF03B5044EC9D
:100CD0000CF0332EF9D762EF02F0060E526E68EC7C
:100CE0000CF0030E0114406E7FEC0CF05DEC01F093
:100CF000356A8FEC0CF03B5044EC0CF05DEC01F0ED
:100D0000080E356E8FEC0CF03B5044EC0CF0332E9B
:100D1000EBD762EF02F00C0E736E070E93EC1BF034
:100D20003B6E030E736E010E93EC1BF0336E406A44
:100D3000526A7FEC0CF0800E216E3B5044EC0CF0BC
:100D40003B5044EC0CF07FEC0CF0400E216E200E7A
:100D5000226E3B5044EC0CF07FEC0CF0030E1B6E4B
:100D60003B5044EC0CF07FEC0CF0600E1B6E3B50E3
:100D700044EC0CF07FEC0CF0030E1C6E3B5044EC8A
:100D80000CF07FEC0CF0100E1E6E100E206E3B501F
:100D900044EC0CF07FEC0CF0020E1E6E020E1F6E87
:100DA0003B5044EC0CF07FEC0CF0100E226E100E59
:100DB0001F6E3B5044EC0CF07FEC0CF0800E226E6A
:100DC000800E1F6E3B5044EC0CF07FEC0CF0200EBC
:100DD0001E6E400E206E3B5044EC0CF07FEC0CF08D
:100DE000020E1D6E010E226E3B5044EC0CF07FECA7
:100DF0000CF0200E1D6E400E1C6E3B5044EC0CF0AF
:100E00007FEC0CF0010E1D6E010E216E3B5044EC88
:100E10000CF07FEC0CF0400E1D6E200E1C6E3B5053
:100E200044EC0CF07FEC0CF0010E1E6E020E216EF5
:100E30003B5044EC0CF07FEC0CF0400E226E200E88
:100E4000216E3B5044EC0CF07FEC0CF0800E1E6EDB
:100E5000800E206E3B5044EC0CF07FEC0CF0400E0A
:100E60001E6E200E206E3B5044EC0CF07FEC0CF01C
:100E7000010E1F6E020E206E3B5044EC0CF07FEC16
:100E80000CF0600E1F6E3B5044EC0CF07FEC0CF04D
:100E9000010E206E3B5044EC0CF0332E4AD762EF2B
:100EA00002F0030E736E010E93EC1BF0336E030E13
:100EB000736E010E93EC1BF0406E526A7FEC0CF0E7
:100EC0005DEC01F0800E21123B5044EC0CF03B50E5
:100ED00044EC0CF05DEC01F0400E2112200E2212C9
:100EE0003B5044EC0CF05DEC01F0030E1B123B5048
:100EF00044EC0CF05DEC01F0600E1B123B5044EC36
:100F00000CF05DEC01F0030E1C123B5044EC0CF0B5
:100F10005DEC01F0100E1E12100E20123B5044EC3E
:100F20000CF05DEC01F0020E1E12020E1F123B507F
:100F300044EC0CF05DEC01F0100E2212100E1F12AA
:100F40003B5044EC0CF05DEC01F0800E2212800E60
:100F50001F123B5044EC0CF05DEC01F0200E1E1211
:100F6000400E20123B5044EC0CF05DEC01F0020E00
:100F70001D12010E22123B5044EC0CF05DEC01F00E
:100F8000200E1D12400E1C123B5044EC0CF05DEC88
:100F900001F0010E1D12010E21123B5044EC0CF029
:100FA0005DEC01F0400E1D12200E1C123B5044EC73
:100FB0000CF05DEC01F0010E1E12020E21123B50EE
:100FC00044EC0CF05DEC01F0400E2212200E2112D8
:100FD0003B5044EC0CF05DEC01F0800E1E12800ED4
:100FE00020123B5044EC0CF05DEC01F0400E1E1260
:100FF000200E20123B5044EC0CF05DEC01F0010E91
:101000001F12020E20123B5044EC0CF05DEC01F07C
:10101000600E1F123B5044EC0CF05DEC01F0010E31
:1010200020123B5044EC0CF0B4EC0CF0640E44EC99
:101030000CF05DEC01F07FEC0CF03B5044EC0CF05C
:10104000332E3CD762EF02F03A0E776E300E766E9A
:10105000040E30EF1BF03A0E776E580E766E040ECB
:1010600030EF1BF03A0E776E800E766E040E30EF86
:101070001BF0030E736E010E93EC1BF0406E526A70
:1010800068EC0CF001501F0B07093B6E030E736EEA
:10109000010E93EC1BF0336E7FEC0CF05DEC01F075
:1010A000010E1C123B5044EC0CF05DEC01F0010E03
:1010B0001D123B5044EC0CF05DEC01F0010E2012CF
:1010C0003B5044EC0CF05DEC01F0010E21123B5062
:1010D00044EC0CF05DEC01F0020E1C123B5044ECB1
:1010E0000CF05DEC01F0100E1E12200E1D123B5094
:1010F00044EC0CF05DEC01F0400E1D12400E1F128E
:101100003B5044EC0CF05DEC01F0200E1C12200E64
:101110001F123B5044EC0CF05DEC01F0100E20125D
:10112000400E1C123B5044EC0CF05DEC01F0600EE4
:101130001B123B5044EC0CF05DEC01F0020E1D1252
:10114000020E1E123B5044EC0CF05DEC01F0010E5F
:101150001E12010E1F123B5044EC0CF05DEC01F02E
:10116000020E2012020E21123B5044EC0CF05DECFA
:1011700001F0010E2212020E1F123B5044EC0CF043
:101180005DEC01F0030E1B123B5044EC0CF05DECE7
:1011900001F0100E2212200E1E123B5044EC0CF0F7
:1011A0005DEC01F0400E2212400E1E123B5044EC4A
:1011B0000CF05DEC01F0200E2012200E21123B50AD
:1011C00044EC0CF05DEC01F0100E1F12400E2012EA
:1011D0003B5044EC0CF05DEC01F0200E2212400E6E
:1011E00021123B5044EC0CF05DEC01F0800E221219
:1011F0003B5044EC0CF05DEC01F0800E1E123B50B5
:1012000044EC0CF05DEC01F0800E20123B5044ECFD
:101210000CF05DEC01F0800E1F123B5044EC0CF022
:101220005DEC01F0800E21123B5044EC0CF0B4EC6C
:101230000CF0640E44EC0CF05DEC01F0332E2CD776
:1012400062EF02F00C0E736E060E93EC1BF03B6E19
:101250007FEC0CF0800E216E400E1B6E3B5044EC78
:101260000CF07FEC0CF0200E226E010E1B6E3B503A
:1012700044EC0CF07FEC0CF0020E1B6E400E216E65
:101280003B5044EC0CF07FEC0CF0200E1B6E800EFB
:10129000216E3B5044EC0CF07FEC0CF0020E1C6E07
:1012A000200E226E3B5044EC0CF07FEC0CF0100E44
:1012B000206E020E1B6E3B5044EC0CF07FEC0CF0E9
:1012C000020E1F6E200E1B6E3B5044EC0CF07FECA8
:1012D0000CF0100E1F6E020E1C6E3B5044EC0CF016
:1012E0007FEC0CF0800E1F6E100E206E3B5044EC15
:1012F0000CF07FEC0CF0400E206E020E1F6E3B5087
:1013000044EC0CF07FEC0CF0010E226E100E1F6E00
:101310003B5044EC0CF07FEC0CF0400E1C6E800E49
:101320001F6E3B5044EC0CF07FEC0CF0010E216E74
:10133000400E206E3B5044EC0CF07FEC0CF0200E85
:101340001C6E010E226E3B5044EC0CF07FEC0CF056
:10135000020E216E400E1C6E3B5044EC0CF07FECF4
:101360000CF0210E216E3B5044EC0CF07FEC0CF0A5
:10137000800E206E200E1C6E3B5044EC0CF07FEC77
:101380000CF0200E206E020E216E3B5044EC0CF04F
:101390007FEC0CF0020E206E200E216E3B5044ECD0
:1013A0000CF07FEC0CF0200E1F6E800E206E3B5078
:1013B00044EC0CF07FEC0CF0210E206E3B5044EC22
:1013C0000CF07FEC0CF0400E1F6E020E206E3B50B6
:1013D00044EC0CF07FEC0CF0210E1F6E3B5044EC03
:1013E0000CF07FEC0CF0400E1E6E010E206E3B5098
:1013F00044EC0CF07FEC0CF0800E1E6E400E1F6E65
:101400003B5044EC0CF07FEC0CF0400E226E010ED1
:101410001F6E3B5044EC0CF07FEC0CF0410E1E6E46
:101420003B5044EC0CF07FEC0CF0400E1D6E800E37
:101430001E6E3B5044EC0CF07FEC0CF0010E1D6E68
:10144000400E226E3B5044EC0CF07FEC0CF0200E72
:101450001D6E010E1E6E3B5044EC0CF07FEC0CF048
:10146000420E1D6E3B5044EC0CF07FEC0CF0200E55
:101470001E6E010E1D6E3B5044EC0CF07FEC0CF028
:10148000800E226E200E1D6E3B5044EC0CF07FEC63
:101490000CF0100E226E020E1D6E3B5044EC0CF050
:1014A0007FEC0CF0220E1E6E3B5044EC0CF07FECF7
:1014B0000CF0100E1E6E800E226E3B5044EC0CF0B1
:1014C0007FEC0CF0010E1C6E100E226E3B5044ECB3
:1014D0000CF07FEC0CF0400E1B6E020E1E6E3B50AB
:1014E00044EC0CF07FEC0CF0010E1B6E100E1E6E27
:1014F0003B5044EC0CF07FEC0CF0400E216E010EE2
:101500001C6E3B5044EC0CF062EF02F03D0E776E27
:10151000280E766E0B0E30EF1BF04380030E736EB9
:10152000000E93EC1BF0406E40500808336E3A0EEC
:10153000776EA80E766E070E30EF1BF03B0E776EBF
:10154000280E766E050E30EF1BF03B0E776E580EB0
:10155000766E040E30EF1BF07FEC0CF0526A030E37
:10156000B8EC0CF0E86A356E8FEC0CF0800E2112AE
:1015700022121E1220121F123B5044EC0CF03B5062
:1015800044EC0CF0219E229E1E9E209E1F9E3B50EE
:1015900044EC0CF0332EEAD762EF02F07FEC0CF053
:1015A000040E346E0F0E356E060E366E800E21124E
:1015B00022121E1220121F12355044EC0CF07FEC48
:1015C0000CF0365044EC0CF0342EF0D7332EE6D726
:1015D00062EF02F0360E776E000E766E0B0E30EF75
:1015E0001BF00150070B526E030EB8EC0CF0C8EC68
:1015F0000CF0330E776E000E766E050E30EF1BF09A
:10160000320E776E000E766E0B0E30EF1BF0050E6D
:10161000736E010E93EC1BF0406E526E070E736EEC
:10162000010E93EC1BF03B6E380EF76E346A5DECE6
:1016300001F0345070EC1BF03B5044EC0CF0342AB9
:10164000330E3464F4D7640E44EC0CF062EF02F015
:10165000030E526EB4EC0CF03A0E776E000E766EFE
:10166000040E30EF1BF0030E526EB4EC0CF03B0E88
:10167000776E000E766E040E30EF1BF0050E526E84
:10168000030E406E030E33125DEC01F03A0EF76E5E
:10169000280EF66E7AEC1BF05DEC01F0B4EC0CF069
:1016A000C8EC0CF0332EF8D762EF02F0010E406E5A
:1016B000040E3326310EF76E09D05DEC01F0680E92
:1016C000F66E7AEC1BF0640E44EC0CF05DEC01F06D
:1016D000700EF66E7AEC1BF0140E44EC0CF05DEC20
:1016E00001F0780EF66E7AEC1BF0140E44EC0CF060
:1016F0005DEC01F0800EF66E7AEC1BF0640E44ECAB
:101700000CF05DEC01F0780EF66E7AEC1BF0140E26
:1017100044EC0CF05DEC01F0700EF66E7AEC1BF010
:10172000140E44EC0CF0332EC8D762EF02F0030E17
:10173000526E0B0EB8EC0CF03C0E776E000E766E0F
:10174000040E30EF1BF0010E406E030E33123C0E00
:10175000F76E5DEC01F0280EF66E7AEC1BF03C0E95
:1017600044EC0CF05DEC01F0300EF66E7AEC1BF000
:10177000280E44EC0CF0332EECD762EF02F0030E8F
:10178000526E0A0EB8EC0CF03D0E776E000E766EBF
:10179000040E30EF1BF03E0E776E000E766E040ED8
:1017A00030EF1BF03E0E776E280E766E040E30EF93
:1017B0001BF0030E526EB4EC0CF03B0E776E800EF5
:1017C000766E040E30EF1BF03B0E776EA80E766E31
:1017D000040E30EF1BF03B0E776ED00E766E010ECE
:1017E00030EF1BF03B0E776EE00E766E020E30EFA0
:1017F0001BF03C0E776E380E766E010E30EF1BF04C
:101800003C0E776E480E766E030E30EF1BF03C0EEA
:10181000776E680E766E010E30EF1BF03C0E776E21
:10182000780E766E010E30EF1BF03C0E776E880E50
:10183000766E010E30EF1BF03C0E776E980E766ED2
:101840000A0E30EF1BF0090E526E0B0EB8EC0CF0C6
:101850003E0E776E500E766E090E30EF1BF03E0E88
:10186000776EA00E766E040E30EF1BF03E0E776E94
:10187000C80E766E020E30EF1BF03E0E776EE00E55
:10188000766E020E30EF1BF03A6E300E626205D0BB
:101890003A66FBD75DEC01F0120062A8E8EF0CF0AD
:1018A000607E62AAFED7060060BE62EF02F05DECC9
:1018B00001F0FF0E1B6E1C6E1D6E1E6E1F6E206EE5
:1018C000216E226E640E3A6E3A66FED762EF02F027
:1018D000016604D0300E65AED624016E006602D0DB
:1018E000450E006E01340118E836013A0038E8462A
:1018F0000118013A010B0036001A013612005DECA6
:1019000001F01B6A1C6A1D6A1E6A1F6A206A216A2E
:10191000226A526A576AE86AB8EC0CF0120035C0C5
:10192000F6FF310EF76E0900F5CF1BF00900F5CF79
:101930001CF00900F5CF1DF00900F5CF1EF00900DD
:10194000F5CF1FF00900F5CF20F00900F5CF21F009
:101950000900F5CF22F0080E3526120000EE02F045
:10196000EE6AE9AEFDD7120068EC0CF000501F0BD8
:10197000040DF3CFF6FF3F0EF76E0900F5CF4FF0E1
:101980000900F5CF50F00900F5CF51F05782120051
:10199000300E626282D75766FBD712005A2A630E56
:1019A0005A64010C5A6A612A5B2A3B0E5B64010C83
:1019B0005B6A5C2A3B0E5C64000C5C6A5D2A0C0E60
:1019C0005D6201D008705D64000C010E5D6E000C5C
:1019D00060846090526A406AE86AB8EC0CF0616A10
:1019E000030E616028D07FEC0CF05DEC01F062A882
:1019F000F7D75D049DEC0DF008B0298E29C021F0C9
:101A000062BA04D0DDEC0CF09AEC0DF062B8F1D7BC
:101A10007FEC0CF097EC0DF05C50BBEC0DF062BA73
:101A200004D02DEC0EF09AEC0DF062A877D0780E71
:101A30006164F2D773D060827FEC0CF0010EB8ECD9
:101A40000CF097EC0DF002049DEC0DF008B2298E1D
:101A500029C021F062BA05D035EC0EF09AEC0DF0F9
:101A6000608062B8F0D77FEC0CF0010EB8EC0CF09F
:101A700097EC0DF00350BBEC0DF062BA04D03FECD4
:101A80000EF09AEC0DF062A804D0780E6164F2D7E3
:101A900045D060827FEC0CF0020EB8EC0CF097ECB5
:101AA0000DF004049DEC0DF008B4298E29C021F03E
:101AB00062BA04D045EC0EF09AEC0DF062B8F1D7A2
:101AC0007FEC0CF0020EB8EC0CF097EC0DF005502A
:101AD000BBEC0DF062BA05D04FEC0EF09AEC0DF0B5
:101AE000608062A804D0780E6164F1D717D060825C
:101AF0007FEC0CF0030EB8EC0CF097EC0DF002EC60
:101B00000EF062BA05D055EC0EF09AEC0DF0608044
:101B100062A804D0780E6164F2D700D097EC0DF083
:101B2000609260B05BEC0EF06090609E120062A864
:101B3000FED7120062AAFED71200080DF3CFF6FFFF
:101B4000320EF76E0900F5CF1BF00900F5CF1CF03F
:101B50000900F5CF1DF00900F5CF1EF00900F5CF03
:101B60001FF00900F5CF20F00900F5CF29F009009A
:101B7000F5CF22F0120024EC0EF05E50080DF3CFEA
:101B8000F6FF330EF76E0900F5CF23F00900F5CF0D
:101B900024F00900F5CF25F00900F5CF26F0090063
:101BA000F5CF27F00900F5CF28F00900F5CF29F08F
:101BB0000900F5CF2AF05F50080DF3CFF6FF340E81
:101BC000F76E0900F55023101B6E0900F550241024
:101BD0001C6E0900F55025101D6E0900F5502610E9
:101BE0001E6E0900F55027101F6E0900F5502810D1
:101BF000206E0900F5502910216E0900F5502A10B9
:101C0000226E12000650080DF3CFF6FF350EF76E68
:101C10000900F5CFCBFFF5CF07F01B6A0900F5CF20
:101C20001CF00900F5CF1DF00900F5CF1EF00900EA
:101C3000F5CF1FF00900F5CF20F00900F5CF21F016
:101C40000900F5CF22F012005F6E5E6A0A0E5F5C3B
:101C5000D8A012005F6E5E2AF9D75A6A5B6A5C2AC6
:101C60003B0E5C6412005C6A1200022A0C0E0262D7
:101C700001D0087202641200010E026E1200032AE3
:101C80003B0E03641200036A1200042A0C0E046265
:101C900001D0087404641200010E046E1200052ABB
:101CA0003B0E05641200056A1200062A0E0E066439
:101CB0001200066A1200AA0E0A6E586A090E596EC0
:101CC00000EE02F0EE5076EC0EF0582A592EFAD7BC
:101CD0001200586A090E596E00EE02F0585087EC57
:101CE0000EF0EE6E582A592EF9D71200A6B2FED782
:101CF000A86E58C0A9FFA69EA69CA684F29E550E6B
:101D0000A76EAA0EA76EA682F28EA6941200A96EE6
:0A1D1000A69EA69CA680A850120013
:10300000030CF0FF0FF3FC00FC00230E346EB90E2E
:10301000356E090E366E342EFED7352EFCD7362E81
:04302000FAD71200C9
:103100009C1C1C0C0C0C1C04636363F3F3F3E3F1D1
:10311000632F45C561A3E3600C632B32BAF323919F
:10312000634345C5D751C561632F2B3228A3E3B054
:103130000C4363F3D75105D10003010000010100E6
:103140006063611060110100636363136313030123
:103150006363637373736371636363F3F3F3E3F143
:10316000630300000000C0200042000092500101F3
:103170000020000020A32300000041C141010040C5
:08318000000123320000009061
:1032000000000000800000000000000090000000AE
:10321000000000009200000000000000921000007A
:103220000002000092100000040200009210000052
:103230000C020000921000000C030000921000002D
:103240000C030010921000000C03001292100000FA
:103250000C030012921000100C0300129210009048
:1033000000000000000000001000000000000000AD
:1033100010001000000000009000100000000000ED
:10332000901010000000000090101000000010002D
:10340000000000000000000000000000008000003C
:103410000000000000A000000000000000A200006A
:103420000000000020A200000000000020A3000017
:103430000000000060A300000000000061A3000085
:103440000000004061A30000000000C061A3000074
:10350000F900000000010000F800000008010000C0
:10351000F700080008010000F6000900080100009B
:10352000F500290008010000F4002B00080100004C
:10353000F3002B2008010000F2002B20080100807E
:10354000FA00000004010000FB0000000401040078
:10355000FC00000004010500FD400000040105001E
:10356000FE40000004010501FF4000000441050188
:08357000FF4000008441050149
:10360000000000008000000000000000100000002A
:103610000000000002000000000000000010000098
:103620000002000000000000040000000000000094
:103630000800000000000000000100000000000081
:103640000000001000000000000000020000000068
:1036500000000000000000100000000000000080DA
:103660007A6E070E736E020E93EC1BF0336E436698
:1036700009D0050E736E000E93EC1BF0406E4050A7
:103680000608336E786A00C079F079B20BD07850B2
:1036900074EC1BF062EC1BF0782A7A507864F7D750
:1036A00079B00BD07AC078F0785074EC1BF062ECF3
:1036B0001BF07806FF0E7862F7D7786A332EE5D7CD
:1036C00062EF02F0406603D03B5044EF0CF0300E46
:1036D00062624DEF0CF04166FAD75DEC01F012002A
:1036E000080DF3CFF6FF06D077C0F7FF080DF350B3
:1036F0007624F66E0900F5CF1BF00900F5CF1CF01B
:103700000900F5CF1DF00900F5CF1EF00900F5CF37
:103710001FF00900F5CF20F00900F5CF21F00900D6
:10372000F5CF22F01200726E68EC0CF000C075F05C
:1037300072C074F0754E05D0742A73507464FAD751
:06374000F7D774501200DF
:103800000000000000000000000000000000008038
:103810000000000000000090000000020000009086
:103820000000001200000090000100120000009053
:1038300008010012000000900C010012000000902E
:103840000C030012000000900C0300120010009006
:103850000C030012021000900C03001212100090D2
:103860000C030012921000900C0300129250009072
:103870000C030012925000910C43001292500091E0
:103880000C430012925001910C430012925005918A
:103890000C430012965005910C430012965105916D
:1038A0000C430012D65105910C430012D6510591DC
:1038B0000C430012D75105910C430052D75105918A
:1038C0000C4300D2D75105910C4300D2D75105D1FA
:1038D0000C4300D3D75105D10C4340D3D75105D168
:1038E0000C4341D3D75105D10C4345D3D75105D112
:1038F0000C4345D7D75105D14C4345D7D75105D1B6
:103900004D4345D7D75105D14D4345D7D75145D123
:103910004D4345D7D751C5D14D4345D7D751C5F1B3
:103920004F4345D7D751C5F16F4345D7D751C5F15F
:103930006F4745D7D751C5F16F4F45D7D751C5F11F
:103940006F6F45D7D751C5F16F6F45D7D751C7F1C5
:103950006F6F45D7D751E7F16F6F45D7D7D1E7F1F3
:103960006F6F45D7D7F1E7F16F6F45D7D7F3E7F121
:103970006F6F45D7F7F3E7F16F6F45D7FFF3E7F1C7
:103980006F6F4DD7FFF3E7F16F6F6DD7FFF3E7F17F
:103990006F6F6FD7FFF3E7F16F6F6FF7FFF3E7F12B
:103A00009C1018080C041C00901C1C0C08081004C6
:103A10009C10140404041C049C1C180808081800BA
:103A2000901C1404040C1404030303838383838114
:103A3000000000000000C0200000000090400000D6
:103A40000000000000A02000000000C000000040B6
:103A500000000020000000900C00000000000800A2
:103A6000000C000000080000000000000404040036
:103A70000000080808000000000004040000000422
:103A80000C0000000000C820000004049040000466
:103A90000000080808A02000000000C00404044042
:103AA000000C0020000800900000008080808080D2
:103AB000000000000060007002000003000200012E
:103AC0002040401020000000000301000001010020
:103AD000402020004010000001000200030002000E
:083AE00000000060100060000E
:103B00000C03001292100090004000C0C541050156
:103B1000410145850000C040222E00000080A32006
:103B200000002B2028A300800000000080000080FF
:103B30000000000010000010000000020200000061
:103B40000000001000100000000300000000000052
:103B50000C000000000000008000000000000000D9
:103B60000000100000000000100000000000000035
:103B70000000000000001000001000000000000025
:103B800090FCFFFFFFFF37DFFFB1FFFF6DA7FEFED9
:103B9000FFDFFFFFDB58D8FFFFFFB636BEF6FFBFE3
:103BA000FFFED8C9FFFFFF6BE3FFFFFFFFFFE7FF4B
:103BB000FFE3FFFFFFF7EFFF7FEFFFFFFBFBFBFFE5
:103BC0007FFFE7F7F7FFFFFFEFFFE7FBFFFFFFFBDD
:103BD0009CDFFFFFDF5815DF9CFFBF3EBEFF379F16
:103BE0009CDFBF369E59159FFFBF9D042CA7FF2A5F
:083BF000FF9FDDCD4D01DD6AF0
:103C000022020000921090200070000080C023016A
:103C1000800000C061A30000000073A1000000C08C
:103C2000510100120000C09000402B208C41058102
:103C3000000000C061A3000003030383838383812A
:103C400060606070707060700003018080818180AE
:103C500020404070300060000300020303020201B4
:103C60004020200040700070FFFFFFFFFFFFFFFFBC
:103C7000F3F3F3F3F3F3F3FBFFFFFFFFFFFFFFFFAC
:103C800060606070707060700000000000000000F4
:103C900060606070707060700000008000800000E4
:103CA000000000C021A22040000000C961A72240FE
:103CB000802048C96DA7264080787DC96DA7274020
:103CC000907C7FED6DEF37459C7F7FFFFFFF37D501
:103CD000FC7F7FFFFFFF3FD5FF7F7FFFFFFF3FD5CB
:103CE000FF7F7FFFFFFF7FF5FF7F7FFFFFFFFFF578
:103D00000C03000000000000000E00000000010095
:103D10000000000004010500000009000801000087
:103D20000001050400000000FFFFFFFFFFFF7FFF11
:103D3000FFFFFFFFFFFFBFDFFCFFFFFFFFFFFFFFF6
:103D40009FFFFFFFFFFFF7FFF3FCFFED6DEFFF6F3E
:103D5000F7FBFFDBFFB7EFFBFFB7D9FFFFFFFFFE6E
:103D6000FFEFEEFFFFFFFEFF7FDFB7FFF7FBFBFF7D
:103D7000FFFFFFF69FFAFDFFFFFFFFBFFEDDDFBF86
:083D8000FFFFFF7FFF7FFFFF43
:103E0000410100000000C00000020000921000000C
:103E10000020000000802300000000C041010000DD
:103E200000002320000000800040000080400101CD
:103E30000000000020A300000000418100000040BD
:103E4000000100120000009022020000000080200B
:103E50004000000000000000200000000000000002
:103E60000000000000100000004000000000000002
:103E70000020000000000000000000002000000002
:103E800000000000400000000000400000000000B2
:103E900000002000000000000000001000000000F2
:103EA0000060601060100000606060006000000052
:103EB0006020401060100000604020106010000082
:103EC00060606010001000009010100000001000F2
:103ED00060606010601000000000006010606070A2
:103EE00000030100000101000300020303020201BC
:083EF00000000080808080804A
:103F000000000000400000000040000000004000F1
:103F10004040400020000000002000000000200081
:103F2000202020000A000000000A000000000A0013
:103F30000A0A0A00400040004040000000404000E3
:103F400040280000190D4000330D4000400D3300A3
:103F5000400D1900401A0D0040331A0033400D0087
:103F60001A400D000D401A000D4033000D33400083
:103F70000D1A4000000E3A002B003A003A000E00E5
:103F80000E3A000065BC62EF02F06870FF0E116E21
:103F9000126E136E146E156E166E176E186E196E05
:103FA0006A6A01EE10F0CC0EEE6EEE6EEE6EEE6E04
:103FB000EE6EEE6EEE6EEE6EF00EEE6E6B6A6850AA
:103FC000FDEC1FF01050FDEC1FF03B50FDEC1FF01E
:103FD0003350FDEC1FF00150FDEC1FF00050FDECE4
:103FE0001FF06050FDEC1FF06B50FDEC1FF0070E52
:103FF000FDEC1FF06596AC8AFFD76B263D6E550E23
:104000003DB0010F3DB2040F3DB4100F3DB6400F5F
:10401000346E550E3DB8010F3DBA040F3DBC100F74
:104020003DBE400F3D6E34C0EEFF3DC0EEFF1200BE
:10403000684369727473616D207374537261762082
:104040002E3020356F4379706972686720742E4472
:104050006854726F657032203030203877772E7751
:104060006E7573756175656C656C74636F72696E7E
:104070007363632E2E6F6B75702F6F72656A746336
:0A4080002F7374737261702E706864
:020000040030CA
:0300010008121EC4
:020005008081F8
:060008000FC00FE00F40E5
:00000001FF
